:030000000219FDE5
:03000B000200AA46
:03002B0002015679
:03005B000202E8B6
:030073000202D5B1
:1000800002030406080C10182030406080040608A3
:100090000C10182030406080A0C00003070F1F0D17
:1000A0000D0403060D0502030202C2AFC0D0C0E07A
:1000B000206214E5256009E473E525F4F58AD2622F
:1000C000D0E0D0D0D2AF3285268AC262E526F46075
:1000D00029D0E0D0D0D297D295D293D2AF32D29756
:1000E000D295D293206F0C2065097405D5E0FDE50B
:1000F0007B4290D0E0D0D0D2AF32758A00C28DD290
:100100006201F301B9306805206502C29701B93078
:100110006805206502C29301B9306805206502C2F6
:100120009501B9C29630680A2065077419D5E0FDBB
:10013000C29701B9C29230680A2065077419D5E0E8
:10014000FDC29301B9C29430680A2065077419D5BD
:10015000E0FDC29501B9C2AFC2AD53E6EFC0D0C059
:10016000E0D2D3D2AFC2CEE52A600720744F152A61
:1001700021BD7800790020742EE580307E01F430B6
:10018000E50278FF53DACF207E0343DA20307E0386
:1001900043DA10C2D8C271E580307E01F430E50246
:1001A00079FFC3E89970CB306103752A402074034E
:1001B000752A40885CD270E86003755F0020740D7A
:1001C000E52B6004152B21CD43DA01C2D820700243
:1001D00021E0A85C206102C27020740221DE882226
:1001E0007882B6040385222420CF0AD0E0D0D04301
:1001F000E610D2AD32C2CF053A7802E52A6005306A
:100200007402152AC3E55C94014005755F00412125
:10021000756000756900E55F2401F55F5003755F47
:10022000FF7982B7020D306E1DC3E522943240166D
:10023000854C227982B7030E306E0BC3E5229432CF
:100240004004798E8722C3E5239522600840041577
:100250002341550523D8CA0569E56970021569D59A
:100260006A69756A017808E56B60497805C3E569D4
:10027000956B4057C3E569956C50087801756A0322
:1002800002028FC3E569956D50057801756A01C357
:10029000E5629524401E7982B7040241C0206E14A5
:1002A000852462E569046003856B69756A017523BD
:1002B0003C0202CBE5622850057562FF41C0F56241
:1002C000E5620470067560FF7569FFD0E0D0D04329
:1002D000E610D2AD32C2AF53E67F7592FA7593FF46
:1002E000C260759104D2AF32C2AF53E6EFC2ADC067
:1002F000D0C0E0C0F0D2D3D2AFA8FBA9FCC2D830A6
:100300007102614F53DACF207E0343DA10307E034F
:1003100043DA20D271E580307E01F420E5026126C7
:1003200088278928A13453DACF207E0343DA20308E
:100330007E0343DA10C2D8C271307402A120780063
:10034000E580307E01F430E502A120885CA10853ED
:10035000DACF207E0343DA20307E0343DA10C27105
:10036000206102812853DACF207E0343DA10307EE9
:100370000343DA20C2D8D27188578958C3E895550B
:10038000F8E99556F97B007E087A00C3E8948CE979
:1003900094005005755B00811A882178A2E6A82197
:1003A0006055C3E894C8E994005008E4D2E4FB7AAD
:1003B0000A61F5C3E89468E994015008E4D2E3FBCC
:1003C0007A0F61F5C3E894D0E994025008E4D2E2D0
:1003D000FB7A1E61F5C3E894A0E994055008E4D2C5
:1003E000E1FB7A3C61F5C3E89498E994085008E48D
:1003F000D2E0FB7A787E00C3E89559FCE9955AFD76
:1004000030E70AECF42401FCEDF43400FD755B00E8
:10041000C3EC9AED9E5003755B018859895A855744
:10042000558558567802A108C3E89527F8E995281C
:10043000F9307C0281EC307B0281EC307A0281E57C
:10044000207502814BE9FDE8FC816AE9C313F9E8F4
:1004500013F830790281E5E9C313F9E813F830782D
:100460000281E5E9C313FDE813FC20612CC3EC9481
:0F0470001CED940240028181ED701EC3EC94C814
:10047F0050180529E52970021529C3E529940A505A
:10048F0002A120755C00D270A120E5296002152918
:10049F007400207F037896E624FAFEE43400FFC34D
:1004AF00EC9EFCED9FFD50067800790081ECC3ECCB
:1004BF0094FFED9400400678FF790081ECEC857293
:1004CF00F0A4C5F0A2F733F87900400302050878CD
:1004DF00FF7900020508E9C313F9E813F8307C0E21
:1004EF00E9600278FFC3E81338F8E43400F9C3E891
:1004FF0094FFE99400400278FF885CD2702061027B
:10050F00A120741FF4552F4BF52FC274EB7002D23C
:10051F0074752A40307403752A0A306102A13420A1
:10052F00740353DAFE207403752B20D0F0D0E0D083
:10053F00D0D2AD43E610327901020564790302058A
:10054F0064790A020564791E020564796402056400
:10055F0079C80205647817E4D5E0FDD8FAD9F622F8
:10056F007A147B7802058B7A107B8C02058B7A0DBF
:10057F007BB402058B7A0B7BC802058BE573D5E044
:10058F0001227902E4C292D5E0FDC293D5E0FDD2FB
:10059F0093D5E0FDD292D5E0FDE920E002C297307D
:1005AF00E002C295E573D5E0FDE920E002D2973075
:1005BF00E002D2957496D5E0FDD9C9EAF8D5E0FDF1
:1005CF00D8FBDBB8C29222C37C007D0075F000051A
:1005DF00F0EA33FAEB33FB50F6EB13FBEA13FAC3F3
:1005EF00E9FFE8FEE89AF8E99BF95004EFF9EEF815
:1005FF00B3EC33FCED33FDD5F0DFEDF9ECF822E889
:10060F0089F08A20D2D4F8A9F07B0030F70B7BFF5A
:10061F00F42401F8E9F43400F9E88520F0A4ADF0F2
:10062F00F8E98520F0A4AFF0FEED2EF974003FFA43
:10063F007C04C3EA13FAE913F9E813F8DCF48BF03E
:10064F0030F70AE8F42401F8E9F43400F9E889F006
:10065F00C2D4F8A9F0227882B60403020704C3E5D6
:10066F005C9419401EE52D54067018206E367805DF
:10067F007994E7146007780A1460027812C3E54191
:10068F0098401F306E098564627569FF756A018530
:10069F002224E4F544F545F546F547F548C26E02C8
:1006AF000704D26E7994E7147013E523F43333F90A
:1006BF0013F8E9540104F9E854FE0206F8E714149C
:1006CF007014E523F4333333F913F8E9540304F9C1
:1006DF00E854FC020700E523F433333333F913F8FE
:1006EF00E954070404F9E854F8C39440F8E9940076
:1006FF00F98844894522C3E54113F9E54013F8C34E
:10070F00E54498F8E54599F9500CC3E89480E994CD
:10071F00FF401602073CC3E8947FE99400500302A0
:10072F00073C787F790002073C788079FF884989F8
:10073F004A22E5492546F8E54A3547F9854A20E436
:10074F00300701F43548FA30E709C3EA94F0401551
:10075F0002077AC3EA940F500302077A78FF79FFF2
:10076F007A0F02077A780079007AF0C3E524956151
:10077F00500AC374019524500B020798E54A20E7ED
:10078F000E020798E54A30E706884689478A4822CD
:10079F0078A5E6FAC3E54933F8E54A33F9D10EE90E
:1007AF0030E70BC3E89480E994FF4013E1D2C3E82C
:1007BF00947FE994005002E1D2787F7900E1D278FA
:1007CF008079FFE820E715C3E52398F84009C3E8CF
:1007DF00940140030207F978010207F9E8F42401B4
:1007EF002523F840030207F978FF884B2278A6E605
:1007FF00FAA847A94812060EE930E70CC3E894019E
:10080F00E994FF401602082EC3E894FFE9940050C4
:10081F000302082E78FF790002082E780179FFE98C
:10082F0020E715C3E54B98F84009C3E8940140034E
:10083F000208557801020855E8F42401254BF840C9
:10084F000302085578FF88242278FF20692879A1B0
:10085F00E76023E541601F74FF8541F0848539F01F
:0F086F00306A0375F005A4F8C5F0600278FFC386
:10087E00E895645002A864886322C3E5409440E57D
:10088E00419401E5635003140199046002F563225B
:10089E007883E6F520120F1B75E89012054675E871
:1008AE009030EDFDA8BDA9BE120FC2756E55756FC5
:1008BE0000C3740013FD7455606613FC74552CFC54
:1008CE0074003DFDECFAEDFBC3E89AE99B4014E59C
:1008DE006E2455F56EE56F3400F56FEA2CFAEB3D9C
:1008EE00FB80E5AE6EAF6FC3E56F13F9E56E13F8DF
:1008FE00C3E913F9E813F87A03C3E913F9E813F817
:10090E00DAF7AA201A7009756E00756F0002092EAB
:10091E001AEA6008EE28FEEF39FFDAF88E6E8F6F56
:10092E002275E890227883E6FF30EDF9A8BDA9BEC6
:10093E000570C3E57094084052757000E9FA79A00D
:10094E00E76044EA7007E571601B020967C3E8952A
:10095E00716010E5715006600C140209730460F9A1
:10096E00020973E571F571C3946D401B7561C0C3C7
:10097E0094044013756180C39404400B756140C3A9
:10098E009404400375610075BB0822EFC3940160A7
:10099E001F7455601BC3E894FFE994035012C3E81B
:1009AE00956EE9956F5009E561600C15610209C5F8
:1009BE00E561F460020561A861C3E524985002A8C0
:1009CE0024C3E89562400AA862E562F4600385627A
:1009DE006188258826E570B4070375BB1022743232
:1009EE0079A787F0A4C5F0A2F733F8C3E895614064
:1009FE0002A861882288248825882688642275406A
:100A0E00007541F022C2AF75C820A8CCA9CDAA3A74
:100A1E0030CF010A75C824D2AFAB3BAC3C883B89C2
:100A2E003CC3E89BF8E99C206908F9306602612412
:100A3E00417EAD3D8A3DF9EA9DFA600678FF79FF69
:100A4E004163AE3EAF3F8B3E8C3FA83BA93CC3E813
:100A5E009EF8E99FF9C3E54113FBE54013FAE82A36
:100A6E00F540E93BF54150067540FF7541FF41CB1E
:100A7E00AA40AB41AC40AD417E047F02C3EB94046F
:100A8E00400D1E1FC3EB94084005206A021E1FC3B3
:100A9E00ED13FDEC13FCDEF7C3EA9CFAEB9DFBEFC6
:100AAE006009C3E913F9E813F8DFF7EA28FAEB391E
:100ABE00FB8A408B4150067BFF8B408B41C3EB94EE
:100ACE00025002D2663069047F0341F67892E6FF47
:100ADE00C3E537948240110FC3E53794A040010F50
:100AEE00C3EF940640027F057E02E541C4540FF920
:100AFE00E541C454F0F8E540C4540F28F8C3E89E0D
:100B0E00FAE99400FB4009C3EA9402EB9400500406
:100B1E007A02E4FB6170AA40AB41EBC4FEEAC45416
:100B2E000F4EFCC3EA9CFAEB9400FBC3E813C3130D
:100B3E00F8EA28FAEB3400FB8A408B41C3EB9402AF
:100B4E004002C2667802EBC4FE7B00EAC4540F4E2C
:100B5E00FAC3EA98FA4005C3940250027A027892D8
:100B6E00E6FF3060026170855192855293D26043E8
:100B7E00E680C3E49AF8E49BF930660261FCE8FA79
:100B8E00E9FBD3E913FDE813FC88518952C3EF94B6
:100B9E00036038EF20E00DE82CF8E93DF9ECFAEDB2
:100BAE00FB020BC5E828F8E939F9C3E82402F8E995
:100BBE003400F97AFE7BFFC3EF9403400E8A538B09
:100BCE0054884D894E8C4F8D508130885389548A6C
:100BDE004D8B4E8C4F8D503069127553F07554FFFE
:100BEE00754FF07550FF7551F07552FF8130E8FA70
:100BFE00D3E813FC8851C3EF94036020EF20E00785
:100C0E00E82CF8ECFA811CE8282402F87AFEC3EFEF
:100C1E00940340088A53884D8C4F813088538A4DF7
:100C2E008C4FE568C3335002646BF5683060028107
:100C3E003A753402D26043E680E52D54066034A83E
:100C4E0040A941C3E913F9E813F8C3E913F9E8130E
:100C5E00F8306904E92440F9C2AF53E67F7591007C
:0E0C6E00C3E498F594E499F595759104D2606D
:100C7C0043E680D2AF22D264754300752000306CFD
:100C8C0003752040020CA1D26475430075204030DE
:100C9C006C0375200078017901206620E52D54063F
:100CAC006002C2647914E541C313700104F8C39463
:100CBC001440027814306904781B791B206010E50D
:100CCC0043600C306903D53404D26DA14B914205BD
:100CDC0043E59B5440B52002A13530690908C3E8AF
:100CEC009940011881C820640A08C3E89940028120
:100CFC00A181C8C264C2AF53E67F75910030661201
:100D0C007594007595F8759104D26043E680D2AF66
:100D1C0081A1E5417EFFC3334005C3334001FEC3CF
:100D2C00E49E759400F595A112C3E533940150022D
:100D3C0081A130640281A1D802A14981C8C26DC2CF
:100D4C00AF53E67F75910085539485549575910446
:100D5C00854D92854E93D26043E680D2AFE52D54FB
:100D6C00066008206A020533020D87306D0D206C79
:100D7C000A2064071581158102162B227800306435
:100D8C00027801E53775F007A4F9E5F028F5F0E9EC
:100D9C00A2F013A2F113A2F213F537C39478500307
:100DAC00753778C3E53795384008D265D297D29518
:100DBC00D293306002A1BE854F92855093D260438E
:100DCC00E68022207D16C2AF754202C292D29630C6
:100DDC006202C295D2AF759F13020FBFC2AF7542AC
:100DEC0002C292D294306202C297D2AF759F1302A4
:100DFC000FBF307243207D20C2AF75420390013487
:100E0C00757B04D295C294306204C293C11CD292F9
:100E1C00D2AF759F10020FBFC2AF75420390013461
:100E2C00757B04D297C296306204C293C13CD292B5
:100E3C00D2AF759F11020FBF207D17C2AF75420351
:100E4C0090010FD295306202C293D2AF759F1002FF
:100E5C000FBFC2AF75420390010FD297306202C22E
:100E6C0093D2AF759F11020FBF207D16C2AF754292
:100E7C0004C296D294306202C293D2AF759F110213
:100E8C000FBFC2AF754204C294D296306202C293B5
:100E9C00D2AF759F10020FBF307243207D20C2AFBE
:100EAC00754205900123757B40D293C29230620447
:100EBC00C297C1C2D296D2AF759F13020FBFC2AFF9
:100ECC00754205900145757B10D293C29230620435
:100EDC00C295C1E2D294D2AF759F13020FBF207D91
:100EEC0017C2AF754205900105D293306202C297CA
:100EFC00D2AF759F13020FBFC2AF75420590011997
:100F0C00D2933062EBC295D2AF759F13020FBF2004
:100F1C007D16C2AF754206C294D292306202C2975D
:100F2C00D2AF759F10020FBFC2AF754206C296D2E8
:100F3C0092306202C295D2AF759F11020FBF307210
:100F4C0044207D20C2AF754201900145757B10D2C3
:100F5C0097C296306204C295E168D294D2AF759F65
:100F6C0011020FBFC2AF754201900123757B40D2B5
:100F7C0095C294306205C297020F89D296D2AF7592
:100F8C009F10020FBF207D17C2AF7542019001194F
:100F9C00D297306202C295D2AF759F11020FBFC2B9
:100FAC00AF754201900105D295306202C297D2AF63
:100FBC00759F10C26522900103757B00D297D29564
:100FCC00D293C296C294C292C262227880760708EB
:100FDC0076070876010876040876FF0876FF08760F
:100FEC0009087602087601087601788C7601087675
:100FFC00000876B40876FF0876FF0876FF087603BB
:10100C000876FF0876010876FF0876250876D00862
:10101C0076780876C80876040876FF087601087694
:10102C000008767A08760A087601087601087600B8
:10103C000876FF087600227887E6FFC2727888C2AD
:10104C007DE630E102D27DC27E7889E630E102D2C3
:10105C007EC3EF94026008758E01D2730210707516
:0F106C008E00C273227880E6149000809378A5DE
:10107B00F67881E6149000809378A6F67886E614CD
:10108B0090008D9378A7F6789FE6F87005756B0046
:10109B0001B7C3E8941140027811E82828F56B25B5
:1010AB006B256B28F56C256B2828F56D7886E6F596
:1010BB0039C394025003753902789CE67538FFB436
:1010CB0002037538A0B4030375388278A3E6149035
:1010DB00009A93F566120FC222227896E6FA789759
:1010EB00E6FB7888E6B40305C3EB940EFB307F0474
:1010FB007A007BFFC3EB9AFCC3948250027C82750F
:10110B0072000572EC8572F0A4C3E5F0947D40F299
:10111B0022D27F11E51205551205557A007B007C12
:10112B001012054BE55C2AFA74003BFBDCF37C04E4
:10113B00C3EB13FBEA13FADCF7FEC27F11E5227552
:10114B007C00757D00E5EF20E603752000052090FF
:10115B003FFFE520146006901DFF146000930460B0
:10116B000375EF1653D9BF7581C043FF8012054637
:10117B0075EF0643B203E5B3240220E70DF521E535
:10118B00E320E0068521B343E301120FC27580FF14
:10119B0075A40075F1B275D4DF7590A975A5FC75B2
:1011AB00F2FE75D50175A60175E241120FC2E4F886
:1011BB00F6D8FD756801120FD712168278988673D0
:1011CB00753001C2AF12055F12056F12055512057E
:1011DB007612055512057D1205551217B512055FCE
:1011EB0012055F12055AC2AF757C00757D0078FA47
:1011FB0079FA308507D9FBD8F7021C00114311711E
:10120B0011E411E578988673120FC27588107589F1
:10121B000275C82475910475D84075A82275B8025B
:10122B0075E690759B80759D0075D10E75BC5875D4
:10123B00BB0875BA1175E880120546D2AF12089E2D
:10124B0075360053DACF207E0343DA20307E03431A
:10125B00DA1043DA01C2D8C27112055FD2617B0387
:10126B007A0CE55B70077A0CDB030211F112055562
:10127B002070030211F1C270E55CC3940240E1E5FA
:10128B002F541F855E5DF55EB55DD5DAD5C2615312
:10129B00DACF207E0343DA20307E0343DA10C2D844
:1012AB00C27178A2E67008D274E52F54E0F52FC214
:1012BB007575290012055A307409C3E529940A4043
:1012CB0002D27512054B78023074027800C3E55CCC
:1012DB009840F0C2AF12056F12056F12056FD2AFB7
:1012EB0012055F754C0012054B788CE6C3940150C8
:1012FB00030213DEE530C3940150030213DE757C49
:10130B00A5757DF1207435C3E55C94FF5003021382
:10131B00DEC2AF120584D2AF12055AC3E55C94014D
:10132B0050EFC2AF12056F12055012056FD2AF12FC
:10133B00055AC3E55C94FF40E902183A7F05D27F5A
:10134B0011E512055AC2AFC27F11E5AE5CC3E55C75
:10135B00947FD2AF500261EE120546C2AF120584E4
:10136B00D2AFDFDA311CC3EE94057897F612055F26
:10137B001217BD7F0AD27F11E512055AC2AFC27F89
:10138B0011E5AE5CC3E55C947FD2AF50E612054627
:10139B00C2AF12056F12055012056FD2AFDFD631F7
:1013AB001CEE24037896F6F87997E7C394824003F2
:1013BB00985006E824827897F612055F1216D01221
:1013CB0017EC12055A11E5C3E55C94FF5002610955
:1013DB0002183A757C00757D00C3E55C954C4003A3
:1013EB00855C4C12055A78017988E7B403027805BD
:1013FB00C3E55C98400241F1C2AF1205841205842B
:10140B00120584D2AF12055F753000E4F531F53269
:10141B000531E531F4703F0532789AE6781914609E
:10142B0012783214600D787D14600878FA1460031A
:10143B00753200C3E53298401D120FC212054615D6
:10144B003275310078998673C2AF120584D2AF78AA
:10145B0098867312055A120550E52A7005307402EE
:0F146B0021F178012074027806C3E55C9840A156
:10147A0012055AE52A70030211F1C2AF120FC2E433
:10148A00F522F523F524F525F526F567D2AF7885FB
:10149A00E6C333F565E4F544F545F546F547F54801
:1014AA00F570F52CF52DF53775700875BB1012051A
:1014BA004612092F30EDFDA8BDA9BEE97001F888D2
:1014CA007112093375700875BB101143C2AF75618B
:1014DA00FF1209EC852261852262852263D2AF75EB
:1014EA002201752401752501752601856069756AD1
:1014FA00017888E6B40307C27D307602D27DD268CD
:10150A00D269753300120F1B120F4A120A0C120A03
:10151A0013120A0C120A13120A0C120C9312066501
:10152A00120D88120DCF120A13120C82306E03129A
:10153A000705206603120858306603120888120D40
:10154A0088120DFE120A13120C93306E0312074111
:10155A00120D88120E75120A13120C82306E0312C3
:10156A00079F120D88120EA4120A13120C93306EE2
:10157A00031207FC120D88120F1B120A1312092FED
:10158A00120C82120D88120F4A120933120A1330F2
:10159A00692C856461856462856069756A01791858
:1015AA007A0CC3E533994009C269D26A8A350215B1
:1015BA00C8C3E55C94014003021524021633306A5D
:1015CA0025206C22E535147006C26AD26BA124F577
:1015DA0035C3E55C940140030215247888E6C39478
:1015EA00036003021633753600C3E55F94014009B0
:1015FA00856462856069756A0178FA79A4E7600290
:10160A007803C3E55F985021307404E52A601A789C
:10161A00F0306C058564617820C3E541985002A1D9
:10162A00240536E55C6002C136753600C2AF120F7A
:10163A00C27887E6FE760211437887EEF6E4F52251
:10164A00F523F524F525F526F565752C00752D008D
:10165A00D2AF12055A120FC278A4E66006C297C228
:10166A0093C295307406E52A700221F1788DE6C39B
:10167A009401400241CE8116901A0D782012171259
:10168A00E520B4A50CA3121712E520B45A030216DA
:10169A00B0757CA5757DF1120FD71216D0757C0036
:1016AA00757D000216CF901A0378807B0A121712F2
:1016BA00A308DBF9901A0F788C7B19121712A3086A
:1016CA00DBF9901A2822C2AF121755121732901A54
:1016DA0000740E121717A37409121717A3741512A0
:1016EA001717901A0378807B0A121716A308DBF9DA
:1016FA00901A0F788C7B19121716A308DBF91217A8
:10170A0068121746901A2822E493F622E6438F01BC
:10171A00538FFDFFC3E583941C400122EF857CB7FC
:10172A00857DB7F0538FFE22438F02438F01857C5C
:10173A00B7857DB7901A0DF0538FFC22901A0D745D
:10174A00A5F117901A0E745AF117227A3079D078C7
:10175A0020901A40F112E520F709A3DAF7227A302D
:10176A0079D0901A40E7F11709A3DAF922AB74A8E5
:10177A0075BB01027980BB02027981BB03027982BF
:10178A00BB04027994BB05027983BB06027986BB46
:10179A0007027992BB08027987BB0902799CBB0AC6
:1017AA00027988BB0B027989E8F7227C0512055F6A
:1017BA00DCFB22C2AF12056F12057612057D1205F7
:1017CA008412055012056F12057612057D120584E2
:1017DA0012055012056F12057612057D120584D284
:1017EA00AF22C2AF12058412057D12057612056F6B
:1017FA0012055012058412057D12057612056F1224
:10180A00055012058412057D12057612056FD2AFB6
:10181A0022AE74AF75C2AF12056F12056F12056F53
:10182A00120550DEF2120584120550DFF8D2AF22FB
:10183A001217BD1217B51217B575740175750175B2
:10184A007600111B7C05AD5C12055FC3ED955C70DB
:10185A00F5C3E55C9401400AC3E55C94FF40370296
:0D186A00187D1217771216D01217BDC2AFED
:1018770075EF161217B5DCD10576C3E576940350DC
:101887000280C21217B50575E5741490009F93F88E
:1018970008C3E57598500280A91217B51217B50548
:1018A70074C3E574940C50028095120FD71216D0AA
:0818B700C2AF75EF161217B560
:0319FD0002114A8A
:101A00000E091507070104FFFF09020101A55A018C
:101A100000B4FFFFFF03FF01FF25D078C804FF01DA
:091A200000FF0A010100FF00FFB4
:101A4000235475726E69677933304123202020203A
:101A500023424C48454C4923463333302320202031
:101A60002020202020202020202020202020202076
:101C0000C2AFC2D353D9BF7581C043B20343FF8073
:101C1000752438752503B1DC7529A5752AF175E29F
:101C20004043F12053A4DF75D4FFD2857DFA7803B9
:101C300079E67C10752200752300901DE97B0675FE
:101C400024987525013085028145208508D8FBD967
:101C5000F9DCF781B7308508D8FBD9F9DCF781B713
:101C6000B19CE493A3C39A6004DDC381B7DBDBB10D
:101C70008E6002812E7B08E493FAA3B16FDBF87AC1
:101C800030B16F752200752300B18EEAFCEBFDC305
:101C9000ED94FE400EB18E8A278B28ED30E0048A49
:101CA000828B83B18E7AC270D8C3ED94FE601950D6
:101CB000CEBD002BEC600F7520007521FF7529004B
:101CC000752A000200008100A827A9280809D80465
:101CD000D90281DCB192EA89AAF281CE0D81A3C337
:101CE000ED94035053EDA2E092007AC5C3E58294CF
:101CF00000E583941C508A200010438F02438F011B
:101D00008529B7852AB7F0300029A827A92808090E
:101D1000438F01538FFDD804D902A133C3E58394C7
:101D20001C4003A3A11689AAE28529B7852AB7F02A
:101D3000A3A116538FFC817F7AC1BD030CE493A34A
:101D4000FAB153DCF8B14B817F8181AA22AB23B178
:101D50006FEBFAEA6222752608C3E52313F523E543
:101D60002213F52250066323A0632201D526EAB18F
:101D7000DCB1DC75260AEAF4200102D285300102CA
:101D8000C285B1DCC3134002C201D526EB22B19259
:101D9000EAFB208502A192308502A197752608AE44
:101DA00024AF25C3EF13FFEE13FEB1E0B1DCC3EAAD
:101DB000133085024480FA30E703632201C3E52330
:101DC00013F523E52213F52250066323A0632201B5
:101DD000D526D9E52265236523F52222AE24AF2539
:101DE0000E0FDEFEDFFCD20122424C48656C6934E6
:071DF000373164F3300601F6
:00000001FF
